:020000040000FA
:04000000D1303A2899
:08000800A000030EA100831209
:1000100005191028831601178312B23081002B288E
:1000200083160113831203140B190310A80DA90DD5
:10003000AA0DAB0DAC0DAC16FF302C02031D2B2806
:10004000FA302B02031D2B2831152A08AF0029088E
:10005000AE002808AD008B100B11210E8300A00EFE
:04006000200E090065
:0C007400203084008001840A80300402E7
:10008000031C3C281230B000E32183160C30850598
:1000900087018312850187010730990000309A009B
:1000A000103083168E008312603083168F00831207
:1000B0000030831691009F008312C83083168100A0
:1000C000831231309000003083168C008312103080
:1000D0008B00562381018E018F010B118B100B10A9
:1000E0008C018B17812031198420B30B7F280310DA
:1000F00085190314B90DF030390203193F219923F2
:10010000722864003210080031110130B7008B13DF
:100110002030370783169B001C141A088312A40092
:100120001030370783169B001C141A088312A30093
:10013000A6000230A6060030370783169B001C1469
:100140001A088312A200A7000130A7068B17321CE1
:10015000AF2822090339A200A309A409A50924088C
:100160002F02031D392923082E02031D39292208D5
:100170002D02031D392901303702031DC4283D1803
:10018000C4283D143E14FE2102303702031DCD2841
:10019000BD18CD28BD143E14102203303702031DB4
:1001A000D6283D19D6283D153E14222204303702A8
:1001B000031DDF28BD19DF28BD153E14342205308C
:1001C0003702031DE8283D1AE8283D163E14462252
:1001D00006303702031DF128BD1AF128BD163E1462
:1001E000572207303702031DFA283D1BFA283D1716
:1001F0003E14682208303702031D0329BD1B032962
:10020000BD173E14792209303702031D0C295E18F0
:100210000C295E143E148A220A303702031D152968
:10022000DE181529DE143E14A3220B303702031DFD
:100230001E295E191E295E153E14BC220C303702A1
:10024000031D2729DE192729DE153E14D1220D3082
:100250003702031D30295E1A30295E163E14E6224D
:100260000E303702031D3929DE1A3929DE163E14F5
:10027000FB22B70A0F303702031808008728013025
:10028000B600B300B400B500B70085018701B11313
:100290008120B30B8F29031085190314B90DF03099
:1002A00039020319B629B40B8F290130370203191B
:1002B00010230230370203191523033037020319C4
:1002C0001A230430370203191F230530370203199C
:1002D0002423063037020319292307303702031974
:1002E0002E2308303702031933230930370203194C
:1002F00038230A30370203193D230B303702031924
:1003000042230C303702031947230D3037020319FB
:100310004C230E303702031951239630B400311D9F
:1003200048293111321C99292D090339AD00AE0934
:10033000AF092F1C48298E018F010C1C48290C1075
:100340002E1E48298B1320303707BB002F08BA0018
:10035000CE2110303707BB002E08BA00CE21003066
:100360003707BB002D08BA00CE218B178501870106
:10037000B70AB6010F303702031C4829562308007C
:100380003E1C08003E101030BB003D08BA00CE21D4
:100390003030BB005E08BA00CE2108008B133A084B
:1003A00083161C159A0083123B0883169B00553058
:1003B0009D00AA309D009C1464009C18DC291C112F
:1003C00083128B170800831610309B001C141A0828
:1003D0008312BD00831630309B001C141A08831250
:1003E000DE00FF30C800CA15CB15CC15CD15CE15D3
:1003F000CF15D015D115D215D31508000130BD0584
:100400000030DE054030C405C0000030C200C60028
:100410004030C505C1000030C300C7005F100800B0
:100420000230BD050030DE050830C405C0000030D4
:10043000C200C6004030C505C1000030C300C7007F
:100440005F1008000430BD050030DE050830C4052B
:10045000C0000030C200C6004030C505C1004030B9
:10046000C300C7005F1008000830BD050030DE057E
:100470008830C405C0000030C200C6000030C50589
:10048000C1000030C300C7005F1008001030BD0578
:100490000030DE058830C405C0008030C200C600D0
:1004A0000030C505C1000030C300C700080020307F
:1004B000BD050030DE051030C405C0000030C200AC
:1004C000C6000030C505C1000030C300C7000800E9
:1004D0004030BD050030DE052030C405C0000030CE
:1004E000C200C6000030C505C1000030C300C7000F
:1004F00008008030BD050030DE052030C405C00096
:100500002030C200C6000030C505C1000030C30065
:10051000C70008000030BD05C130DE0508304418B2
:10052000013AC418023AC405C00000304618013A26
:10053000C618023AC200C6008030C505C1000030AE
:10054000C300C70008000030BD05C230DE0508301A
:100550004418013AC418023AC405C00000304618D5
:10056000013AC618023AC200C6008030C505C10073
:100570008030C300C70008000030BD05C430DE0570
:100580000A30C405C0000030C200C6000030C51BE0
:10059000803AC505C1000030C71B803AC300C700C0
:1005A00008000030BD05C830DE050A30C405C000B3
:1005B0000230C200C6000030C51B803AC505C1002C
:1005C0000030C71B803AC300C70008000030BD05DB
:1005D000D030DE050930C405C0000030C200C600BE
:1005E0000030C51B803AC505C1000030C71B803AEA
:1005F000C300C70008000030BD05E030DE0509304B
:10060000C405C0000130C200C6000030C51B803ADE
:10061000C505C1000030C71B803AC300C7000800F1
:10062000003085061130870608000230850610303C
:100630008706080002308506103087060800023061
:1006400085062030870608000230850620308706A0
:100650000800003085060230870608000030850655
:10066000043087060800003085060430870608003D
:1006700002308506083087060800023085060830FB
:1006800087060800223085060030870608002230E1
:100690008506003087060800123085060030870680
:1006A0000800123085060030870608003D18FE213C
:1006B000BD1810223D192222BD1934223D1A4622AE
:1006C000BD1A57223D1B6822BD1B79225E188A2263
:1006D000DE18A3225E19BC22DE19D1225E1AE622A0
:1006E000DE1AFB220800B601B301B4013C1C7B2BCF
:1006F000BC01BC147D2BBC013C143C08B60064005A
:10070000812B822B832B842B852BFF30B41B850000
:10071000B41F8501B30B7F2BB40B7F2B0310B60CDA
:10072000B608031D7F2B0030BB003C08BA00CE2169
:1007300008008F08031908008F0178308E00C80F59
:10074000C32DC80A441CC92B461CBA2BCA1CAB2B90
:10075000CA014A15D72B4A1DB02BCA01CA15D72B7F
:10076000CA1DB52BCA014A16D72B4A1ED72BCA0160
:10077000CA14D72B4A1DBF2BCA014A16D72BCA1D34
:10078000C42BCA014A16D72B4A1ED72BCA01CA143A
:10079000D72BCA1CCE2BCA014A15D72B4A1DD32BE7
:1007A000CA01CA15D72B4A1ED72BCA014A15C41C29
:1007B000FE2BC61CEF2BCB1CE02BCB014B150C2CBE
:1007C0004B1DE52BCB01CB150C2CCB1DEA2BCB0104
:1007D0004B160C2C4B1E0C2CCB01CB140C2C4B1D94
:1007E000F42BCB014B160C2CCB1DF92BCB014B164C
:1007F0000C2C4B1E0C2CCB01CB140C2CCB1C032C27
:10080000CB014B150C2C4B1D082CCB01CB150C2C04
:100810004B1E0C2CCB014B15441D332C461D242C98
:10082000CC1C152CCC014C15412C4C1D1A2CCC0188
:10083000CC15412CCC1D1F2CCC014C16412C4C1E30
:10084000412CCC01CC14412C4C1D292CCC014C1634
:10085000412CCC1D2E2CCC014C16412C4C1E412C75
:10086000CC01CC14412CCC1C382CCC014C15412C87
:100870004C1D3D2CCC01CC15412C4C1E412CCC01E7
:100880004C15C41D692CC61D5A2CCD1C4B2CCD01FA
:100890004D155F13772C4D1D502CCD01CD15772CA8
:1008A000CD1D552CCD014D16772C4D1E772CCD012D
:1008B000CD14772C4D1D5F2CCD014D16772CCD1D01
:1008C000642CCD014D16772C4D1E772CCD01CD1407
:1008D000772CCD1C6E2CCD014D15772C4D1D732C16
:1008E000CD01CD15772C4D1E772CCD014D155F1BFD
:1008F000A02C441EA02C461E912CCE1C822CCE0176
:100900004E15AE2C4E1D872CCE01CE15AE2CCE1D15
:100910008C2CCE014E16AE2C4E1EAE2CCE01CE141B
:10092000AE2C4E1D962CCE014E16AE2CCE1D9B2C01
:10093000CE014E16AE2C4E1EAE2CCE01CE14AE2CD9
:10094000CE1CA52CCE014E15AE2C4E1DAA2CCE01D0
:10095000CE15AE2C4E1EAE2CCE014E15C41ED52C7F
:10096000C61EC62CCF1CB72CCF014F15E32C4F1D34
:10097000BC2CCF01CF15E32CCF1DC12CCF014F16BE
:10098000E32C4F1EE32CCF01CF14E32C4F1DCB2CB7
:10099000CF014F16E32CCF1DD02CCF014F16E32CE7
:1009A0004F1EE32CCF01CF14E32CCF1CDA2CCF0148
:1009B0004F15E32C4F1DDF2CCF01CF15E32C4F1E1D
:1009C000E32CCF014F15441F0A2D461FFB2CD01CD2
:1009D000EC2CD0015015182D501DF12CD001D01544
:1009E000182DD01DF62CD0015016182D501E182D84
:1009F000D001D014182D501D002DD0015016182DE7
:100A0000D01D052DD0015016182D501E182DD001C7
:100A1000D014182DD01C0F2DD0015015182D501D9D
:100A2000142DD001D015182D501E182DD0015015A1
:100A3000C41F3F2DC61F302DD11C212DD1015115B2
:100A40004D2D511D262DD101D1154D2DD11D2B2DF3
:100A5000D10151164D2D511E4D2DD101D1144D2DC9
:100A6000511D352DD10151164D2DD11D3A2DD101DC
:100A700051164D2D511E4D2DD101D1144D2DD11C8E
:100A8000442DD10151154D2D511D492DD101D115A7
:100A90004D2D511E4D2DD1015115451F752D471F4F
:100AA000662DD21C572DD2015215DF13832D521DF6
:100AB0005C2DD201D215832DD21D612DD20152168B
:100AC000832D521E832DD201D214832D521D6B2DE6
:100AD000D2015216832DD21D702DD2015216832DB4
:100AE000521E832DD201D214832DD21C7A2DD20115
:100AF0005215832D521D7F2DD201D215832D521EEA
:100B0000832DD2015215DF1BAC2DC51FAC2DC71F85
:100B10009D2DD31C8E2DD3015315BA2D531D932D0E
:100B2000D301D315BA2DD31D982DD3015316BA2D49
:100B3000531EBA2DD301D314BA2D531DA22DD301A8
:100B40005316BA2DD31DA72DD3015316BA2D531EFC
:100B5000BA2DD301D314BA2DD31CB12DD301531503
:100B6000BA2D531DB62DD301D315BA2D531EBA2D50
:100B7000D3015315C0214008C4004108C5005F18C7
:100B8000DF145F1CDF104808C9000C304A05031D44
:100B900005120C304B05031D85120C304C05031D4E
:100BA00005100C304D05031D85100C304E05031D3E
:100BB00087100C304F05031D07110C305005031D25
:100BC00007100C305105031D87120C305205031D10
:100BD00007120C305305031D871149080E02031834
:100BE0001D2E12304A05031D051612304B05031D3C
:100BF000851612304C05031D051412304D05031DDA
:100C0000851412304E05031D871412304F05031D45
:100C1000071512305005031D071412305105031D2E
:100C2000871612305205031D071612305305031D97
:100C30008715FF304802031908008F08031D0800BC
:100C4000812049080E02031C1D2E18304A05031D81
:100C5000051206304A05031D051618304B05031D05
:100C6000851206304B05031D851618304C05031DF3
:100C7000051006304C05031D051418304D05031DE5
:100C8000851006304D05031D851418304E05031DD3
:100C9000871006304E05031D871418304F05031DBD
:100CA000071106304F05031D071518305005031DA9
:100CB000071006305005031D071418305105031D99
:100CC000871206305105031D871618305205031D83
:100CD000071206305205031D071618305305031D71
:0C0CE000871106305305031D871508001E
:084000000A00030005000500A1
:02400E00CC33B1
:10420000010078007A007C007E007B0079007F004E
:104210007D007A0078007E007C007D007F007900C0
:104220000200F200F600FA00FE00F200F600FA00CA
:10423000FE00F200F600FA00FE00F200F600FA00BE
:10424000FF00050005000500050009000900090040
:1042500009000D000D000D000D00110011001100EE
:104260000100FF00FF00FF00FF00FF00FF00FF0054
:10427000FF00FF00FF00FF00FF00FF00FF00FF0046
:10428000FF007B00FF00FF00FF00FF00FF00FF00BA
:10429000FF00FF00FF00FF00FF00FF00FF00FF0026
:1042A000FF00FE00FF00FF00FF00FF00FF00FF0017
:1042B000FF00FF00FF00FF00FF00FF00FF00FF0006
:1042C000FF001100FF00FF00FF00FF00FF00FF00E4
:1042D000FF00FF00FF00FF00FF00FF00FF00FF00E6
:1042E000FF00FF00FF00FF00FF00FF00FF00FF00D6
:1042F000FF00FF00FF00FF00FF00FF00FF00DD00E8
:00000001FF
